
 Start         Length Name               Class

  0001:0000    0C4BH  _TEXT              CODE
  0002:0000    02FEH  MEM_TEXT           CODE
  0003:0000    0000H  _FARDATA           FAR_DATA
  0003:0000    0000H  _FARBSS            FAR_BSS
  0003:0000    0010H  NULL               BEGDATA
  0003:0010    0270H  _DATA              DATA
  0003:0280    0004H  _FPSEG             DATA
  0003:0284    0000H  _CVTSEG            DATA
  0003:0284    0000H  _SCNSEG            DATA
  0003:0284    0000H  _CONST             CONST
  0003:0284    0006H  _INIT_             INITDATA
  0003:028A    0000H  _INITEND_          INITDATA
  0003:028A    0000H  _EXIT_             EXITDATA
  0003:028A    0000H  _EXITEND_          EXITDATA
  0003:028A    0046H  _BSS               BSS
  0003:02D0    0000H  _BSSEND            BSSEND


Detailed map of segments

 0001:0000 0164 C=CODE   S=_TEXT          G=(none)  M=c0d.ASM    ACBP=48
 0001:0164 0096 C=CODE   S=_TEXT          G=(none)  M=RANDINT.C  ACBP=48
 0001:01FA 0024 C=CODE   S=_TEXT          G=(none)  M=ATEXIT     ACBP=48
 0001:021E 0089 C=CODE   S=_TEXT          G=(none)  M=EXIT       ACBP=48
 0001:02A8 0000 C=CODE   S=_TEXT          G=(none)  M=FILES      ACBP=48
 0001:02A8 0000 C=CODE   S=_TEXT          G=(none)  M=FILES2     ACBP=48
 0001:02A8 004B C=CODE   S=_TEXT          G=(none)  M=IOERROR    ACBP=48
 0001:02F4 0011 C=CODE   S=_TEXT          G=(none)  M=ISATTY     ACBP=48
 0001:0306 0029 C=CODE   S=_TEXT          G=(none)  M=LSEEK      ACBP=48
 0001:032F 0017 C=CODE   S=_TEXT          G=(none)  M=N_LXMUL    ACBP=28
 0001:0346 0037 C=CODE   S=_TEXT          G=(none)  M=RAND       ACBP=48
 0001:037E 00AE C=CODE   S=_TEXT          G=(none)  M=SETUPIO    ACBP=48
 0001:042C 0016 C=CODE   S=_TEXT          G=(none)  M=TELL       ACBP=48
 0001:0442 00C6 C=CODE   S=_TEXT          G=(none)  M=FFLUSH     ACBP=48
 0001:0508 0040 C=CODE   S=_TEXT          G=(none)  M=FLUSHALL   ACBP=48
 0001:0548 0154 C=CODE   S=_TEXT          G=(none)  M=FSEEK      ACBP=48
 0001:069C 010F C=CODE   S=_TEXT          G=(none)  M=SETVBUF    ACBP=48
 0001:07AC 0147 C=CODE   S=_TEXT          G=(none)  M=WRITE      ACBP=48
 0001:08F4 0063 C=CODE   S=_TEXT          G=(none)  M=WRITEA     ACBP=48
 0001:0958 0036 C=CODE   S=_TEXT          G=(none)  M=XFFLUSH    ACBP=48
 0001:098E 0026 C=CODE   S=_TEXT          G=(none)  M=FMEMCPY    ACBP=48
 0001:09B4 0047 C=CODE   S=_TEXT          G=(none)  M=FMEMSET    ACBP=48
 0001:09FC 005E C=CODE   S=_TEXT          G=(none)  M=HEAP       ACBP=48
 0001:0A5A 000C C=CODE   S=_TEXT          G=(none)  M=SUBALLOC   ACBP=48
 0001:0A66 0000 C=CODE   S=_TEXT          G=(none)  M=WCFNCPTR   ACBP=48
 0001:0A66 01E5 C=CODE   S=_TEXT          G=(none)  M=FHEAP      ACBP=48
 0002:0000 02A3 C=CODE   S=MEM_TEXT       G=(none)  M=ASMMEM     ACBP=68
 0002:02A3 005B C=CODE   S=MEM_TEXT       G=(none)  M=WINMEM     ACBP=28
 0003:0000 0000 C=FAR_DATA S=_FARDATA       G=DGROUP  M=c0d.ASM    ACBP=68
 0003:0000 0000 C=FAR_BSS S=_FARBSS        G=DGROUP  M=c0d.ASM    ACBP=68
 0003:0000 0010 C=BEGDATA S=NULL           G=DGROUP  M=c0d.ASM    ACBP=68
 0003:0010 003A C=DATA   S=_DATA          G=DGROUP  M=c0d.ASM    ACBP=68
 0003:004A 0000 C=DATA   S=_DATA          G=DGROUP  M=RANDINT.C  ACBP=48
 0003:004A 0002 C=DATA   S=_DATA          G=DGROUP  M=ATEXIT     ACBP=48
 0003:004C 0006 C=DATA   S=_DATA          G=DGROUP  M=EXIT       ACBP=48
 0003:0052 0190 C=DATA   S=_DATA          G=DGROUP  M=FILES      ACBP=48
 0003:01E2 002A C=DATA   S=_DATA          G=DGROUP  M=FILES2     ACBP=48
 0003:020C 005B C=DATA   S=_DATA          G=DGROUP  M=IOERROR    ACBP=48
 0003:0268 0000 C=DATA   S=_DATA          G=DGROUP  M=ISATTY     ACBP=48
 0003:0268 0000 C=DATA   S=_DATA          G=DGROUP  M=LSEEK      ACBP=48
 0003:0268 0000 C=DATA   S=_DATA          G=DGROUP  M=N_LXMUL    ACBP=48
 0003:0268 0004 C=DATA   S=_DATA          G=DGROUP  M=RAND       ACBP=48
 0003:026C 0000 C=DATA   S=_DATA          G=DGROUP  M=SETUPIO    ACBP=48
 0003:026C 0000 C=DATA   S=_DATA          G=DGROUP  M=TELL       ACBP=48
 0003:026C 0000 C=DATA   S=_DATA          G=DGROUP  M=FFLUSH     ACBP=48
 0003:026C 0000 C=DATA   S=_DATA          G=DGROUP  M=FLUSHALL   ACBP=48
 0003:026C 0000 C=DATA   S=_DATA          G=DGROUP  M=FSEEK      ACBP=48
 0003:026C 0004 C=DATA   S=_DATA          G=DGROUP  M=SETVBUF    ACBP=48
 0003:0270 0000 C=DATA   S=_DATA          G=DGROUP  M=WRITE      ACBP=48
 0003:0270 0000 C=DATA   S=_DATA          G=DGROUP  M=WRITEA     ACBP=48
 0003:0270 0000 C=DATA   S=_DATA          G=DGROUP  M=XFFLUSH    ACBP=48
 0003:0270 0000 C=DATA   S=_DATA          G=DGROUP  M=FMEMCPY    ACBP=48
 0003:0270 0000 C=DATA   S=_DATA          G=DGROUP  M=FMEMSET    ACBP=48
 0003:0270 0000 C=DATA   S=_DATA          G=DGROUP  M=HEAP       ACBP=48
 0003:0270 0006 C=DATA   S=_DATA          G=DGROUP  M=SUBALLOC   ACBP=48
 0003:0276 0004 C=DATA   S=_DATA          G=DGROUP  M=WCFNCPTR   ACBP=48
 0003:0280 0000 C=DATA   S=_DATA          G=DGROUP  M=ASMMEM     ACBP=68
 0003:0280 0000 C=DATA   S=_DATA          G=DGROUP  M=FHEAP      ACBP=48
 0003:0280 0004 C=DATA   S=_FPSEG         G=DGROUP  M=c0d.ASM    ACBP=48
 0003:0284 0000 C=DATA   S=_CVTSEG        G=DGROUP  M=c0d.ASM    ACBP=48
 0003:0284 0000 C=DATA   S=_SCNSEG        G=DGROUP  M=c0d.ASM    ACBP=48
 0003:0284 0000 C=CONST  S=_CONST         G=DGROUP  M=c0d.ASM    ACBP=48
 0003:0284 0000 C=INITDATA S=_INIT_         G=DGROUP  M=c0d.ASM    ACBP=48
 0003:0284 0006 C=INITDATA S=_INIT_         G=DGROUP  M=SETUPIO    ACBP=48
 0003:028A 0000 C=INITDATA S=_INITEND_      G=DGROUP  M=c0d.ASM    ACBP=28
 0003:028A 0000 C=EXITDATA S=_EXIT_         G=DGROUP  M=c0d.ASM    ACBP=48
 0003:028A 0000 C=EXITDATA S=_EXITEND_      G=DGROUP  M=c0d.ASM    ACBP=28
 0003:028A 0000 C=BSS    S=_BSS           G=DGROUP  M=c0d.ASM    ACBP=48
 0003:028A 0002 C=BSS    S=_BSS           G=DGROUP  M=RANDINT.C  ACBP=48
 0003:028C 0040 C=BSS    S=_BSS           G=DGROUP  M=ATEXIT     ACBP=48
 0003:02CC 0000 C=BSS    S=_BSS           G=DGROUP  M=IOERROR    ACBP=48
 0003:02CC 0000 C=BSS    S=_BSS           G=DGROUP  M=ISATTY     ACBP=48
 0003:02CC 0000 C=BSS    S=_BSS           G=DGROUP  M=LSEEK      ACBP=48
 0003:02CC 0000 C=BSS    S=_BSS           G=DGROUP  M=SETUPIO    ACBP=48
 0003:02CC 0000 C=BSS    S=_BSS           G=DGROUP  M=WRITEA     ACBP=48
 0003:02CC 0000 C=BSS    S=_BSS           G=DGROUP  M=FMEMCPY    ACBP=48
 0003:02CC 0000 C=BSS    S=_BSS           G=DGROUP  M=FMEMSET    ACBP=48
 0003:02D0 0000 C=BSS    S=_BSS           G=DGROUP  M=ASMMEM     ACBP=68
 0003:02D0 0000 C=BSSEND S=_BSSEND        G=DGROUP  M=c0d.ASM    ACBP=28

  Address         Publics by Name

 0000:0000 idle  GETCURRENTTIME
 0000:0000 idle  GETWINFLAGS
 0002:02A3       GET_TEMP_BLOCK
 0000:0000 idle  GLOBALALLOC
 0000:0000 idle  GLOBALFREE
 0000:0000 idle  GLOBALHANDLE
 0000:0000 idle  GLOBALLOCK
 0000:0000 idle  GLOBALREALLOC
 0000:0000 idle  GLOBALSIZE
 0000:0000 idle  GLOBALUNLOCK
 0002:000E idle  INITMEM
 0001:0000 idle  LibEntry
 0001:0164       LIBMAIN
 0000:0000 idle  LOCALINIT
 0000:0000 idle  LOCKSEGMENT
 0001:032F       N_LXMUL@
 0001:0185       RANDOMINT
 0002:02D3       RLS_TEMP_BLOCK
 0002:02EA       SIZ_TEMP_BLOCK
 0002:0023 idle  STOPMEM
 0000:0000 idle  UNLOCKSEGMENT
 0001:00A5       WEP
 0001:01FA idle  _atexit
 0001:0A2C idle  _calloc
 0003:0010       _errno
 0001:026C idle  _exit
 0001:0442       _fflush
 0001:0508       _flushall
 0001:0A45       _free
 0001:05CA       _fseek
 0001:0646 idle  _ftell
 0002:0065       _GETMEM
 0001:0A5A       _GetSubAllocClientData
 0003:028A idle  _hInst
 0001:02F4       _isatty
 0001:0306       _lseek
 0001:09FC       _malloc
 0001:0357       _rand
 0001:0A11 idle  _realloc
 0002:01E2       _RLSMEM
 0001:069C       _setvbuf
 0002:01CC       _SIZMEM
 0001:0346       _srand
 0003:0270 idle  _SubAllocClientData
 0001:042C       _tell
 0003:0014 idle  __8087
 0000:0000 idle  __acrtused
 0003:004A       __atexitcnt
 0003:028C       __atexittbl
 0001:028D       __cexit
 0001:0099       __checknull
 0001:0087       __cleanup
 0001:029B idle  __c_exit
 0003:020C idle  __doserrno
 0001:02E1 idle  __DOSERROR
 0003:020E idle  __dosErrorToSV
 0001:027B idle  __exit
 0003:004C       __exitbuf
 0003:004E idle  __exitfopen
 0003:0050 idle  __exitopen
 0001:0AAD       __farcallocf
 0001:0B20       __farfreef
 0001:0A66       __farmallocf
 0001:0B52       __farreallocf
 0001:098E       __fmemcpy
 0001:09DA       __fmemset
 0003:0280 idle  __FPVector
 0001:09B4 idle  __fsetmem
 0003:0019 idle  __hInstance
 0001:02A8       __IOERROR
 0003:01E2       __nfile
 0003:01E4       __openfd
 0003:0016 idle  __osmajor
 0003:0017 idle  __osminor
 0003:0018 idle  __osmode
 0003:0016 idle  __osversion
 0003:0012 idle  __protected
 0003:0284 idle  __RealCvtVector
 0001:009A       __restorezero
 0003:0284 idle  __ScanTodVector
 0001:037E       __setupio
 0003:0052       __streams
 0001:009B       __terminate
 0003:0016 idle  __version
 0001:01EC       __WEP
 0003:001B       __WinAllocFlag
 0001:08F4       __write
 0001:0958       __xfflush
 0003:0276 idle  ___ReadBufFPtr
 0001:07AC       ___write
 0003:0278       ___WriteBufFPtr

  Address         Publics by Value

 0000:0000 idle  __acrtused
 0000:0000 idle  LOCALINIT
 0000:0000 idle  LOCKSEGMENT
 0000:0000 idle  UNLOCKSEGMENT
 0000:0000 idle  GETWINFLAGS
 0001:0000 idle  LibEntry
 0000:0000 idle  GETCURRENTTIME
 0000:0000 idle  GLOBALALLOC
 0000:0000 idle  GLOBALFREE
 0000:0000 idle  GLOBALHANDLE
 0000:0000 idle  GLOBALLOCK
 0000:0000 idle  GLOBALREALLOC
 0000:0000 idle  GLOBALSIZE
 0000:0000 idle  GLOBALUNLOCK
 0001:0087       __cleanup
 0001:0099       __checknull
 0001:009A       __restorezero
 0001:009B       __terminate
 0001:00A5       WEP
 0001:0164       LIBMAIN
 0001:0185       RANDOMINT
 0001:01EC       __WEP
 0001:01FA idle  _atexit
 0001:026C idle  _exit
 0001:027B idle  __exit
 0001:028D       __cexit
 0001:029B idle  __c_exit
 0001:02A8       __IOERROR
 0001:02E1 idle  __DOSERROR
 0001:02F4       _isatty
 0001:0306       _lseek
 0001:032F       N_LXMUL@
 0001:0346       _srand
 0001:0357       _rand
 0001:037E       __setupio
 0001:042C       _tell
 0001:0442       _fflush
 0001:0508       _flushall
 0001:05CA       _fseek
 0001:0646 idle  _ftell
 0001:069C       _setvbuf
 0001:07AC       ___write
 0001:08F4       __write
 0001:0958       __xfflush
 0001:098E       __fmemcpy
 0001:09B4 idle  __fsetmem
 0001:09DA       __fmemset
 0001:09FC       _malloc
 0001:0A11 idle  _realloc
 0001:0A2C idle  _calloc
 0001:0A45       _free
 0001:0A5A       _GetSubAllocClientData
 0001:0A66       __farmallocf
 0001:0AAD       __farcallocf
 0001:0B20       __farfreef
 0001:0B52       __farreallocf
 0002:000E idle  INITMEM
 0002:0023 idle  STOPMEM
 0002:0065       _GETMEM
 0002:01CC       _SIZMEM
 0002:01E2       _RLSMEM
 0002:02A3       GET_TEMP_BLOCK
 0002:02D3       RLS_TEMP_BLOCK
 0002:02EA       SIZ_TEMP_BLOCK
 0003:0010       _errno
 0003:0012 idle  __protected
 0003:0014 idle  __8087
 0003:0016 idle  __osversion
 0003:0016 idle  __osmajor
 0003:0016 idle  __version
 0003:0017 idle  __osminor
 0003:0018 idle  __osmode
 0003:0019 idle  __hInstance
 0003:001B       __WinAllocFlag
 0003:004A       __atexitcnt
 0003:004C       __exitbuf
 0003:004E idle  __exitfopen
 0003:0050 idle  __exitopen
 0003:0052       __streams
 0003:01E2       __nfile
 0003:01E4       __openfd
 0003:020C idle  __doserrno
 0003:020E idle  __dosErrorToSV
 0003:0270 idle  _SubAllocClientData
 0003:0276 idle  ___ReadBufFPtr
 0003:0278       ___WriteBufFPtr
 0003:0280 idle  __FPVector
 0003:0284 idle  __ScanTodVector
 0003:0284 idle  __RealCvtVector
 0003:028A idle  _hInst
 0003:028C       __atexittbl


